:100000000C9440050C9487050C9487050C94870587
:100010000C9487050C9487050C9487050C94870530
:100020000C9487050C9487050C94A90C0C947B0DFB
:100030000C94831C0C9487050C9487050C948705FD
:100040000C9487050C9487050C9487050C94870500
:100050000C9487050C94F71C0C9487050C94870569
:100060000C9487050C9487050C9487050C948705E0
:100070000C9487050C9487050C9487050C948705D0
:100080000C9487050C9487050C9487050C948705C0
:100090000C9487050C9487050C9487050C948705B0
:1000A0000C9487050C9487050C948705E80D0A0EBF
:1000B000F80E0A0EF80E4F0E720EF80EC70EDA0E7C
:1000C000F011F0111F121F127D12BB12D514D5149E
:1000D000D412D514D513D513A914D514D514C0141E
:1000E000507C7E8051634F621B7B35198029102C18
:1000F0007F37808059585A5B1D7A78060E8011052B
:10010000343836805C575D5E070479090D3A0B0A76
:100110007D330F3052808080161439150C3C18172F
:1001200080808080808080808080808080808080CF
:100130002E2D2731532A5455201F8021263B24235E
:100140002F1312285F5660611A1E2B08253D1C22B2
:10015000444342454C4E494B80808080413E403F65
:100160004B6579626F6172642073746172742E0AD8
:100170000055534220636F6E666967757265642E21
:100180000A000D0A696E69740A005B445D005B43F6
:100190005D002C0346004300390038003000430066
:1001A000200041006C007400200043006F006E00CE
:1001B000740072006F006C006C006500720000003B
:1001C0000A0354004D004B002E00000004030904F4
:1001D00009028D00050100A032090400000103019D
:1001E00001000921110100012240000705810308D7
:1001F000000A0904010001030102000921110100A4
:1002000001224D000705820308000A0904020001CB
:1002100003000000092111010001223600070583B7
:100220000308000A09040300020300000009211169
:1002300001000122220007058403200001070504B4
:10024000032000010904040001030000000921113A
:100250000100012239000705850320000112011069
:100260000100000008EDFE0C9800010102000105EC
:10027000010906A101050719E029E71500250195E7
:100280000875018102050819012905950575019177
:10029000029501750391010507190029F71500253D
:1002A0000195F875018102C00631FF0974A10109A9
:1002B00075150026FF009520750881020976150046
:1002C00026FF00952075089102C005010980A10153
:1002D000850216810026B7001A81002AB700751022
:1002E00095018100C0050C0901A1018503160100DB
:1002F000269C021A01002A9C02751095018100C0FB
:1003000005010902A1010901A10005091901290539
:10031000150025019505750181029501750381017F
:100320000501093009311581257F9502750881067F
:1003300009381581257F950175088106050C0A3855
:10034000021581257F950175088106C0C005010948
:1003500006A101050719E029E71500250195087593
:10036000018102950175088101050819012905958A
:100370000575019102950175039101050719002981
:10038000FF150026FF00950675088100C0636F6E9B
:1003900073756D65723A20253034580A007379738D
:1003A00074656D3A20253034580A000A0025303231
:1003B0005820006B6579626F6172643A20004C4589
:1003C000443A20253032580A00253032583A202548
:1003D0003031366225730A00722F63203031323398
:1003E0003435363738394142434445460A0064655E
:1003F0006C5F6B65795F6269743A2063616E277424
:100400002064656C3A20253032580A006164645FCC
:100410006B65795F6269743A2063616E277420614D
:1004200064643A20253032580A004F6E6573686F55
:10043000743A2074696D656F75740A00290A002585
:1004400075002F002575005D28002564002000251B
:100450006400200025640020002564007C00253015
:100460003258006D6F7573656B6579205B62746ED1
:100470007C782079207620685D287265702F616312
:100480006C293A205B006D6B5F776865656C5F7403
:10049000696D655F746F5F6D6178203D2025640A2A
:1004A000006D6B5F776865656C5F6D61785F737019
:1004B000656564203D2025640A006D6B5F74696D7D
:1004C000655F746F5F6D6178203D2025640A006D63
:1004D0006B5F6D61785F7370656564203D20256496
:1004E0000A006D6B5F696E74657276616C203D20E9
:1004F00025640A006D6B5F64656C6179203D202581
:10050000640A006D6B5F776865656C5F74696D6523
:100510005F746F5F6D6178203D2025640A006D6B0C
:100520005F776865656C5F6D61785F737065656442
:10053000203D2025640A006D6B5F74696D655F74F2
:100540006F5F6D6178203D2025640A006D6B5F6DE3
:1005500061785F7370656564203D2025640A006DD5
:100560006B5F696E74657276616C203D2025640A4C
:10057000006D6B5F64656C6179203D2025640A0025
:100580000A00257500363A20776865656C5F7469E6
:100590006D655F746F5F6D61783A20000A002575A4
:1005A00000353A20776865656C5F6D61785F7370C0
:1005B0006565643A20000A00257500343A207469A4
:1005C0006D655F746F5F6D61783A20000A00257574
:1005D00000333A206D61785F73706565643A20007E
:1005E0000A00257500323A20696E74657276616C76
:1005F000286D73293A20000A00257500313A2064DD
:10060000656C6179282A31306D73293A20000A0916
:100610002D2056616C756573202D0A004D3E004DEE
:1006200025643E20003F0073657420646566617533
:100630006C740A00433E200077686572652064652B
:100640006C74613A20637572736F723D25642C205F
:10065000776865656C3D25640A5365652068747428
:10066000703A2F2F656E2E77696B697065646961CA
:100670002E6F72672F77696B692F4D6F7573655F8A
:100680006B6579730A000A092D204D6F7573656BD0
:100690006579202D0A4553432F713A0971756974A4
:1006A0000A313A0964656C6179282A31306D732901
:1006B0000A323A09696E74657276616C286D732925
:1006C0000A333A096D61785F73706565640A343A7C
:1006D0000974696D655F746F5F6D61780A353A09F9
:1006E000776865656C5F6D61785F73706565640AD6
:1006F000363A09776865656C5F74696D655F746F1C
:100700005F6D61780A0A703A097072696E742076BA
:10071000616C7565730A643A097365742064656673
:1007200061756C74730A75703A092B310A646F77BE
:100730006E3A092D310A706775703A092B31300A0B
:100740007067646F776E3A092D31300A0A737065ED
:100750006564203D2064656C7461202A206D617899
:100760005F7370656564202A202872657065617406
:10077000202F2074696D655F746F5F6D6178290A41
:10078000003F004D3E2000433E20004C25640A00FF
:100790000A092D20436F6E736F6C65202D0A455337
:1007A000432F713A09717569740A6D3A096D6F7555
:1007B00073656B65790A000A092D204D61676963CD
:1007C000202D0A643A0964656275670A783A0964FB
:1007D00065627567206D61747269780A6B3A0964A5
:1007E00065627567206B6579626F6172640A6D3A44
:1007F000096465627567206D6F7573650A763A09DD
:1008000076657273696F6E0A733A097374617475F1
:10081000730A633A09636F6E736F6C65206D6F6462
:10082000650A302D343A096C61796572302D3428AF
:100830004631302D4634290A506175733A09626F8A
:100840006F746C6F616465720A6E3A094E4B524F59
:100850000A003F004E4B524F3A206F66660A004E28
:100860004B524F3A206F6E0A0074696D65725F7269
:10087000656164333228293A202530346C580A00E7
:100880006B6579626F6172645F6E6B726F3A20257F
:10089000580A006B6579626F6172645F69646C65A8
:1008A0003A2025580A006B6579626F6172645F7047
:1008B000726F746F636F6C3A2025580A00686F730B
:1008C000745F6B6579626F6172645F6C65647328D5
:1008D000293A2025580A000A092D2053746174759D
:1008E00073202D0A004743433A20342E392E3220FC
:1008F0004156522D4C4942433A20312E382E307306
:10090000766E204156525F415243483A20617672DA
:10091000350A004F5054494F4E533A204C554641EA
:10092000204D4F5553454B45592045585452414B46
:10093000455920434F4E534F4C4520434F4D4D4159
:100940004E44204E4B524F204B45594D41505F5322
:10095000454354494F4E20343039360A00425549F8
:100960004C443A2063646634623531202831313A90
:1009700031393A32372041707220323720323031EB
:1009800038290A005649443A2030784645454428DB
:10099000544D4B2E29205049443A20307839383074
:1009A000432846433938304320416C7420436F6EEE
:1009B00074726F6C6C657229205645523A203078FB
:1009C000303130300A00444553433A20544D4B2EC9
:1009D000206B6579626F617264206669726D776100
:1009E000726520666F72204643393830430A000A28
:1009F000092D2056657273696F6E202D0A000A6DED
:100A00006F7573653A206F66660A000A6D6F7573BD
:100A1000653A206F6E0A000A6B6579626F617264D5
:100A20003A206F66660A000A6B6579626F617264CC
:100A30003A206F6E0A000A6D61747269783A206F0D
:100A400066660A000A6D61747269783A206F6E0AF0
:100A5000000A64656275673A206F6E0A000A646571
:100A60006275673A206F66660A000A0A626F6F74E1
:100A70006C6F616465722E2E2E2000433E200000B4
:100A800011241FBECFEFDAE0DEBFCDBF04B603FEF8
:100A900027C08091A2029091A302A091A402B091DC
:100AA000A5028730904BA740B04BD1F41092A20220
:100AB0001092A3021092A4021092A50214BE84B751
:100AC000877F84BF0FB6F894A895809160008861F5
:100AD00080936000109260000FBEE0E0F8E309959B
:100AE00011E0A0E0B1E0E4E0FBE402C005900D926B
:100AF000A833B107D9F722E0A8E3B1E001C01D9205
:100B0000A23AB207E1F70E94CC090C9480250C941C
:100B10000000FF93EF93E0913801F0913901309795
:100B200009F00995EF91FF910895FC0185918030BE
:100B300011F0EFDFFBCF0895FF27E0E230E247FF3F
:100B40000CC0419597FF09C0EDE2609570958095C6
:100B50009095611D711D811D911D27FF02C021957A
:100B600030E350E2AA27660F771F881F991FAA1F3C
:100B7000A41710F0A41B63955A95A9F7AA3008F0A2
:100B8000A95FA05DAF93F39561157105810591058E
:100B900041F7ED3211F4EF93F395F21718F43F9308
:100BA000F395FBCF8F91B5DFFA95E1F70895E991C1
:100BB000F9918591803021F0853219F0AADFF9CFC3
:100BC000089520E0E89455915532C1F3503311F463
:100BD000689455915A3348F4505390F3220F022EE3
:100BE000220F220F200D250FF4CF0EF421958991AD
:100BF0009991533619F3533729F1533559F1BC0103
:100C000088279927E8945C3621F489919991689412
:100C10005591543639F446EF7EF077FF0DC08FEFD3
:100C20009FEF0AC055374AE039F0583540E121F0CE
:100C3000523642E009F00895FF93EF937DDFEF9184
:100C4000FF91B7CFFF93EF93FC0181918030B9F30F
:100C500060DFFBCFFF93EF9368DFF1CFDF93CF939C
:100C6000CDB7DEB72596A3DFCF91DF91089584B18C
:100C70008F6084B93E98469A3F9A8AB1806F8AB94C
:100C80005F9A479884B1806784B985B1806785B9D8
:100C9000EAE4F1E01192119281E0EA35F807D1F728
:100CA000EAE3F1E01192119281E0EA34F807D1F71A
:100CB0008AE491E090935D0180935C018AE391E086
:100CC00090935B0180935A010895AF92BF92DF9297
:100CD000EF92FF920F931F93CF93DF9380915A016E
:100CE00090915B0120915C0130915D0130935B013B
:100CF00020935A0190935D0180935C0100E010E025
:100D0000C1E0D0E085B1807F802B85B9BE01002E87
:100D100002C0660F771F0A94E2F75B01A094B094BB
:100D200040E050E08BB1282F2F78CA0134E0880FC3
:100D3000991F3A95E1F7822B8BB92AE02A95F1F7B2
:100D400000C0CA01880F991FA0915A01B0915B01A0
:100D5000A80FB91F2D913C9126233723232B09F08F
:100D6000479AE5E3EA95F1F70000D6B45F98FAE018
:100D7000FA95F1F700C0A0915C01B0915D017D0191
:100D8000E80EF91EF701369B05C0208131812A212A
:100D90003B2104C020813181262B372B31832083D6
:100DA00026B5ED2CF12C2D1518F026B530E004C039
:100DB00026B530E021503F4F2E193F09263031052E
:100DC00068F020915A0130915B01280F391FF90119
:100DD00020813181A80FB91F2D933C93FAE1FA9538
:100DE000F1F700C047985F9A20EA2A95F1F74F5F24
:100DF0005F4F4830510509F095CFA0915C01B0914B
:100E00005D01E0915A01F0915B0150962D913C916A
:100E10005197808991892817390751F00E94C11C88
:100E200060935E0170935F01809360019093610114
:100E30000F5F1F4F0031110509F064CF81E0DF9192
:100E4000CF911F910F91FF90EF90DF90BF90AF90E7
:100E5000089520915C0190915D01E22FF92FE80F38
:100E6000F11DE80FF11D80819181089580FF02C07E
:100E70002C9A01C02C9881FF02C02D9A01C02D9898
:100E800082FF02C02E9A08952E98089580918601BF
:100E900008959FB7F894109265019FBF90919902B1
:100EA000943009F057C09091E9009F703091EC00A8
:100EB000232F217030FD20E8922B24E02093E900BD
:100EC0002091EB0020FF43C02091EE0027FF3FC0A0
:100ED00020916201222321F02091E80025FF37C0F4
:100EE0001092620126E03091E80035FD15C0309186
:100EF0009902343061F53091EB0035FD28C0215066
:100F000021F481E08093620122C0EFE9FFE0319794
:100F1000F1F700C00000E7CF8093F1008091E80076
:100F200085FD0AC08091E80080FFFCCF8091E80039
:100F30008E778093E80006C08FB7F89421E0209365
:100F400065018FBF9F709093E90080E008959F70C6
:100F50009093E9008FEF0895CF93DF9300D01F9215
:100F6000CDB7DEB79C0180919902843019F593E0EA
:100F700099833B832A839093E9008FEF9091E80057
:100F8000815095FD06C095ED9A95F1F7000081110D
:100F9000F5CF8091E80085FF0DC040E050E063E0B0
:100FA00070E0CE0101960E94990A8091E8008E7748
:100FB0008093E8000F900F900F90DF91CF910895EC
:100FC000CF93DF9300D01F92CDB7DEB72091990267
:100FD000243021F522E029839B838A8383E0809358
:100FE000E9008FEF9091E800815095FD06C095EDE6
:100FF0009A95F1F700008111F5CF8091E80085FF07
:101000000DC040E050E063E070E0CE0101960E9428
:10101000990A8091E8008E778093E8000F900F90F6
:101020000F90DF91CF910895209199022430F1F42F
:1010300022E02093E9002FEF3091E800215035FDA8
:1010400006C035ED3A95F1F700002111F5CF20915A
:10105000E80025FF0BC040E050E065E070E00E9432
:10106000990A8091E8008E778093E8000895CF93E5
:10107000DF9320919902243009F048C0EC0180915F
:101080000A018823E1F080910B018823C1F085E0FB
:101090008093E9008FEF9091E800815095FD06C0A4
:1010A0009AE29A95F1F700C08111F5CF8091E8009E
:1010B00085FF2CC040E050E060E270E017C081E0A6
:1010C0008093E9008FEF9091E800815095FD06C074
:1010D00095ED9A95F1F700008111F5CF8091E80028
:1010E00085FF14C040E050E068E070E0CE010E944F
:1010F000990A8091E8008E778093E80080E2FE01F3
:10110000A6E6B1E001900D928A95E1F7DF91CF91CB
:1011100008958EE891E00E949505809198028111D2
:1011200009C00E942E0C0E948B0C8091E20084600A
:101130008093E20008958AE891E00E94950510925C
:10114000980208950895209163012F5F822F62E332
:101150000E944625992319F0209363010895109267
:10116000630180916501882371F180919902843037
:1011700041F58091E9008F702091EC00922F9170E1
:1011800020FD90E8892B94E09093E9009091EB008A
:1011900090FF14C09091EE0097FF10C09091E8006E
:1011A00095FF03C01092F100F9CF9091E80090FFF5
:1011B00005C09091E8009E779093E8008F7080932F
:1011C000E90010926501089542E061EC81E00E941F
:1011D000A80B42E061EC82E00E94A80B42E061ECC7
:1011E00083E00E94A80B42E261EC84E00E94A80B1D
:1011F00042E261EC85E00C94A80B80919B02833065
:1012000009F455C030F4813071F0823009F48EC099
:1012100008958A3009F47AC08B3009F460C08930AF
:1012200009F09CC020C080919A02813A09F096C0D2
:101230008091E800877F8093E80080919E029091E2
:101240009F02892B21F460E286E691E003C060E012
:1012500080E090E070E00E94E40A8091E8008B77E3
:101260008093E800089580919A02813209F076C057
:1012700080919E0290919F02009719F0049709F0C7
:101280006DC08091E800877F8093E8008091E8003E
:1012900082FD05C0809199028111F8CF5FC08091D5
:1012A000F100809386018091E8008B7753C0809194
:1012B0009A02813A09F052C080919E0290919F0259
:1012C000892B09F04BC08091E800877F8093E8006C
:1012D0008091E80080FFFCCF80910A0136C08091A8
:1012E0009A028132D9F580919E0290919F02892BBA
:1012F000A9F58091E800877F8093E8000E94DD0BCC
:1013000080919C0280930A010C94F71480919A02B8
:10131000813221F58091E800877F8093E8000E9468
:10132000DD0B80919D0280938701089580919A0240
:10133000813AA1F48091E800877F8093E800809152
:10134000E80080FFFCCF809187018093F1008091BD
:10135000E8008E778093E8000C94DD0B08950895E3
:10136000089580918601809364011092860180E047
:101370000E9436070E9492100C94F7140C94B10945
:101380000E94411C80919702882329F00E946A1CC8
:1013900081110C94830A089584B7877F84BF0FB6A8
:1013A000F894A89580916000886180936000109205
:1013B00060000FBE90E080E80FB6F8948093610063
:1013C000909361000FBE89E497E00E94F81B82E8C9
:1013D00091E00E9495050E94AF090E94D10F0E94E2
:1013E0002E0C0E948B0C8091E20084608093E200BE
:1013F0007894809199028430E1F781ED97E001972C
:1014000039F0EFE9FFE03197F1F700C00000F7CFC6
:1014100081E791E00E9495050E94D30F80E091E062
:101420000E94100F80E691E00E9495050E94B0098D
:1014300080919902853019F40E94C009F9CF0E9469
:10144000D70FF6CF0E947F1C8091640180938601A4
:1014500008950C94220A292F332723303105C9F02F
:1014600064F42130310581F02230310509F043C0A8
:101470008DE890E020ED31E042C021323105F1F0FD
:101480002232310541F137C082E190E02DE532E0B2
:1014900036C099278130910541F08230910541F0A5
:1014A000892B49F5ECECF1E005C0E0ECF1E002C07D
:1014B000E2E9F1E0849190E09F0121C06530D8F429
:1014C000E62FF0E0EE0FFF1FED5DFE4F2081318132
:1014D00089E090E014C0653070F470E0FB01EE0F1D
:1014E000FF1FE75EFE4F20813181FB01EC5EFE4F66
:1014F000808190E004C080E090E020E030E0FA01DC
:1015000031832083089580E189BD82E189BD09B4DA
:1015100000FEFDCF8091D8008F7D8093D800809110
:10152000E00082608093E0008091E00081FDFCCFCC
:101530000895CF92DF92EF92FF920F931F93CF9374
:10154000DF93EC018B016A010E94FC0B811133C017
:10155000C114D10439F0F60180819181081B190B67
:10156000C80FD91FE12CF12C0115110519F180913B
:10157000E80085FD16C08091E8008E778093E80032
:10158000C114D10449F0F60180819181E80EF91E61
:10159000F182E08285E00FC00E94FC0B882321F3DA
:1015A0000AC089918093F10001501109FFEFEF1AF1
:1015B000FF0ADACF80E0DF91CF911F910F91FF906A
:1015C000EF90DF90CF9008952091A0023091A1027A
:1015D0002617370748F06115710539F42091E800A6
:1015E0002E772093E80001C0B90140E06115710534
:1015F000A9F120919902222309F443C0253009F46E
:1016000042C02091E80023FD40C02091E80022FD67
:1016100032C02091E80020FFE9CF4091F3002091F3
:10162000F20030E0342BFC01CF016115710559F057
:101630002830310540F481918093F10061507109A7
:101640002F5F3F4FF1CF41E02830310509F040E0F6
:101650002091E8002E772093E800C8CF4111C9CF30
:101660000AC080919902882361F0853061F08091F1
:10167000E80083FD0AC08091E80082FFF2CF80E09D
:10168000089582E0089583E0089581E0089520910F
:10169000A0023091A1022617370748F061157105A5
:1016A00039F42091E8002E772093E80001C0B901B9
:1016B000FC0120E06115710591F180919902882368
:1016C00009F440C0853009F43FC08091E80083FDF3
:1016D0003DC08091E80082FD2FC08091E80080FF2E
:1016E000E9CF2091F3008091F20090E0922B6115F8
:1016F000710559F08830910540F424912093F10050
:101700003196615071090196F2CF21E0089709F0F6
:1017100020E08091E8008E778093E800CBCF211104
:10172000CCCF0AC080919902882361F0853061F0A6
:101730008091E80083FD0AC08091E80082FFF2CF2B
:1017400080E0089582E0089583E0089581E008959F
:10175000982F973058F59093E900981739F07091C9
:10176000EC002091ED005091F00003C0242F762F63
:1017700050E021FF19C03091EB003E7F3093EB0029
:101780003091ED003D7F3093ED003091EB00316002
:101790003093EB007093EC002093ED005093F00039
:1017A0002091EE0027FF07C09F5FD3CF8F708093FB
:1017B000E90081E0089580E0089580919A0287FF12
:1017C00011C08091E80082FD05C0809199028111CD
:1017D000F8CF11C08091E8008B770BC080919902FF
:1017E000882349F08091E80080FFF8CF8091E800DD
:1017F0008E778093E80008952091E4003091E50011
:1018000095E64091EC00842F817040FF22C08091CA
:10181000E80080FD1CC080919902882391F08530FA
:1018200091F08091EB0085FD10C04091E400509153
:10183000E5004217530729F39A01915011F784E00C
:10184000089582E0089583E0089581E0089580E09E
:1018500008954091E80042FFDECF08950E949C0C5D
:101860000E94A40CE0EEF0E0808181608083E8EDCE
:10187000F0E080818F77808319BCA7EDB0E08C9178
:101880008E7F8C9380818F7E808310929802089542
:101890000F931F93CF93DF930E949C0C0E94A40C84
:1018A000C8EDD0E088818F778883888180688883BD
:1018B00088818F7D888319BC1092990210929502BD
:1018C000109297021092960200EE10E0F8018081CB
:1018D0008B7F808388818160888342E060E080E044
:1018E0000E94A80BE1EEF0E080818E7F8083E2EE23
:1018F000F0E0808181608083808188608083F8014E
:1019000080818E7F8083888180618883DF91CF9101
:101910001F910F910895E8EDF0E080818F7E808324
:10192000E7EDF0E080818160808384E082BF81E028
:10193000809398020C94480CE8EDF0E080818E7F53
:1019400080831092E20008951092DA001092E10074
:1019500008951F920F920FB60F9211242F933F9369
:101960004F935F936F937F938F939F93AF93BF93A7
:10197000EF93FF938091E10082FF0BC08091E20022
:1019800082FF07C08091E1008B7F8093E1000E947D
:10199000A3088091DA0080FF1FC08091D80080FFEB
:1019A0001BC08091DA008E7F8093DA008091D9008D
:1019B00080FF0DC080E189BD82E189BD09B400FED0
:1019C000FDCF81E0809399020E94890805C019BC6F
:1019D000109299020E949B088091E10080FF19C03B
:1019E0008091E20080FF15C08091E2008E7F80939D
:1019F000E2008091E20080618093E2008091D80053
:101A000080628093D80019BC85E0809399020E947F
:101A1000BE098091E10084FF30C08091E20084FF24
:101A20002CC080E189BD82E189BD09B400FEFDCFF3
:101A30008091D8008F7D8093D8008091E1008F7EC7
:101A40008093E1008091E2008F7E8093E20080919C
:101A5000E20081608093E20080919502882311F07A
:101A600084E007C08091E30087FD02C081E001C0EF
:101A700083E0809399020E94290A8091E10083FF0C
:101A800029C08091E20083FF25C08091E100877F1B
:101A90008093E10082E080939902109295028091F8
:101AA000E1008E7F8093E1008091E2008E7F809341
:101AB000E2008091E20080618093E20042E060E019
:101AC00080E00E94A80B8091F00088608093F00075
:101AD0000E94A208FF91EF91BF91AF919F918F91CA
:101AE0007F916F915F914F913F912F910F900FBE1A
:101AF0000F901F9018951F920F920FB60F921124FE
:101B00002F933F934F935F936F937F938F939F9305
:101B1000AF93BF93CF93DF93EF93FF93C091E9000F
:101B2000CF708091EC00D82FD17080FDD0E810925A
:101B3000E9008091F000877F8093F00078940E9404
:101B4000BF0D1092E9008091F00088608093F00052
:101B5000CD2BCF70C093E900FF91EF91DF91CF9132
:101B6000BF91AF919F918F917F916F915F914F91B5
:101B70003F912F910F900FBE0F901F9018951F93BC
:101B8000CF93DF93CDB7DEB7AA970FB6F894DEBF39
:101B90000FBECDBFEAE9F2E088E08E0F9091F10030
:101BA00091938E13FBCF0E94FD088091E80083FF84
:101BB0001FC180919A0290919B02492F50E04A30B8
:101BC000510508F015C1FA01EA5AFF4F0C94662539
:101BD000803881F0823809F00BC180919E028F70AD
:101BE0008093E9008091EB0085FB882780F91092B3
:101BF000E90006C08091960290919702911182604F
:101C00009091E800977F9093E8008093F100109204
:101C1000F100C8C0282F2D7F09F0EAC0882319F0F1
:101C2000823061F0E5C080919C02813009F0E0C013
:101C3000933009F080E0809397022BC080919C0242
:101C4000811127C080919E028F7009F4D1C08093CA
:101C5000E9002091EB0020FF1CC0933021F480911B
:101C6000EB00806214C09091EB0090619093EB00C8
:101C700021E030E0A90102C0440F551F8A95E2F728
:101C80004093EA001092EA008091EB008860809314
:101C9000EB001092E9008091E800877F86C08111F7
:101CA000A7C010919C021F778091E3008078812B60
:101CB0008093E3008091E800877F8093E8000E9492
:101CC000DD0B8091E80080FFFCCF8091E30080680D
:101CD0008093E300111102C082E001C083E0809391
:101CE000990286C08058823008F082C080919C02A0
:101CF00090919D028C3D53E0950779F583E08A83AE
:101D00008AE289834FB7F894DE01139620E03EE023
:101D100051E2E32FF0E050935700E49120FF03C01D
:101D2000E295EF703F5FEF708E2F90E0EA3010F099
:101D3000C79601C0C0968D939D932F5F243149F7BC
:101D40004FBF8091E800877F8093E8006AE270E0EF
:101D5000CE0101960E94E40A14C0AE014F5F5F4FAE
:101D600060919E020E942B0ABC01892B09F440C09D
:101D70009091E800977F9093E80089819A810E9472
:101D8000470B8091E8008B778093E80031C0803862
:101D900079F58091E800877F8093E8008091950233
:101DA0008093F1008091E8008E778093E8000E9494
:101DB000DD0B1EC081111CC090919C029230C0F4BA
:101DC0008091E800877F8093E800909395020E94BD
:101DD000DD0B80919502811106C08091E30087FDA3
:101DE00002C081E001C084E0809399020E94E4086F
:101DF0008091E80083FF0AC08091E800877F80938C
:101E0000E8008091EB0080628093EB00AA960FB609
:101E1000F894DEBF0FBECDBFDF91CF911F91089523
:101E200090938D0180938C010895E0918C01F09145
:101E30008D01309721F00190F081E02D099480E030
:101E40000895EF92FF920F931F93CF93DF93E0914A
:101E50008C01F0918D013097B1F18C010280F381FA
:101E6000E02D09958091840282FF2DC080FF04C07F
:101E700083EB93E00E949505E80110E28DEAE82EDD
:101E800083E0F82E8091840280FF0BC088811F922E
:101E90008F93FF92EF920E942E060F900F900F905B
:101EA0000F90115021961111EDCF8091840280FF87
:101EB0000AC08BEA93E0DF91CF911F910F91FF90C1
:101EC000EF900C949505DF91CF911F910F91FF90AA
:101ED000EF900895E0918C01F0918D01309721F001
:101EE0000480F581E02D09940895CF93DF93EC01F0
:101EF00080918A0190918B01C817D90709F1D0937D
:101F00008B01C0938A01E0918C01F0918D01309793
:101F1000B9F00680F781E02DCE0109958091840209
:101F200082FF0EC080FF0CC0DF93CF938DE993E05A
:101F30009F938F930E942E060F900F900F900F90FB
:101F4000DF91CF910895CF93DF93EC0180918801C9
:101F500090918901C817D90709F1D0938901C093DD
:101F60008801E0918C01F0918D013097B9F00084E7
:101F7000F185E02DCE0109958091840282FF0EC08B
:101F800080FF0CC0DF93CF938DE893E09F938F93F6
:101F90000E942E060F900F900F900F90DF91CF911F
:101FA00008950C9493100E94AC1C0C9437068F92E9
:101FB0009F92AF92BF92CF92DF92EF92FF920F93D8
:101FC0001F93CF93DF9300D000D01F92CDB7DEB721
:101FD0000E9465060FE811E0F12C8F2D0E94290761
:101FE0004C01F801A080B180A826B926A114B10443
:101FF00039F4F3940E5F1F4FF8E0FF12EECF39C0B3
:102000008091840281FD0E949410E12CCC24C39421
:10201000D12CC6018A219B21892B21F1E982FA82E8
:1020200021E0C60188219921892B09F420E02B8326
:102030000E94B51C8160782F9D838C8349815A81D1
:102040006B818D810E94CA1049815A816B817C818C
:102050008D810E942E1CF801808191818C259D2507
:1020600091838083E394CC0CDD1CF0E1EF12D1CF9F
:10207000C0CF8FEF89838A831B820E94B51C816049
:10208000782F9D838C8349815A816B818D810E9439
:10209000CA100E942D1C0E94761F10918E010E9472
:1020A000150F181759F10E94150F80938E0190910A
:1020B000840292FF0EC090FF0CC01F928F938EEB94
:1020C00093E09F938F930E942E060F900F900F9096
:1020D0000F9080918E010F900F900F900F900F90A6
:1020E000DF91CF911F910F91FF90EF90DF90CF90F4
:1020F000BF90AF909F908F900C943F1C0F900F90CB
:102100000F900F900F90DF91CF911F910F91FF9043
:10211000EF90DF90CF90BF90AF909F908F900895F9
:102120000C94360708950895EF92FF920F931F9332
:10213000CF93DF9388ED93E00E949505C0E0D0E057
:102140008DE2E82E81E0F82E09EC13E08C2F0E943E
:1021500029070E94131CFF92EF929F938F93DF93A6
:10216000CF931F930F930E942E0621968DB79EB793
:1021700008960FB6F8949EBF0FBE8DBFC830D1052C
:1021800029F7DF91CF911F910F91FF90EF90089564
:1021900008950895CF93DF93CDB7DEB72B970FB691
:1021A000F894DEBF0FBECDBF942F4F83252F5887E5
:1021B00069877A878B874A855B85452B21F02F3F7E
:1021C00009F59F3FF9F4DE01119686E0FD011192B9
:1021D0008A95E9F785E0FE01379601900D928A9580
:1021E000E1F749815A816B817C818D819E810E94BA
:1021F000DC172B960FB6F894DEBF0FBECDBFDF9174
:10220000CF9108954F81588569857A858B850E9485
:102210002E1CD9CFCF93882309F465C0C82F8CEF2B
:102220008C0F813A20F080E58C0F8E3248F48C2F91
:102230000E94C022811157C08C2F0E94B41A0CC07A
:1022400080E28C0F883058F4C77081E001C0880F9D
:10225000CA95EAF70E945F1BCF910C94A31B8BE5F4
:102260008C0F833078F4C53A29F0C63A31F083E810
:1022700090E005C081E890E002C082E890E0CF9154
:102280000C94750F88E58C0F853168F5C83A89F094
:10229000C93A91F0CA3A99F0CB3AA1F0CC3AA9F0F8
:1022A000CD3AB1F0CE3AB9F0CF3AC1F080E090E04B
:1022B00017C082EE90E014C089EE90E011C08AEE63
:1022C00090E00EC085EB90E00BC086EB90E008C07C
:1022D00083EB90E005C084EB90E002C087EB90E0D8
:1022E000CF910C94A30FCF910895882349F19CEFCF
:1022F000980F913A20F090E5980F9E3218F40E94C2
:10230000071B0DC090E2980F983058F4877091E049
:1023100001C0990F8A95EAF7892F0E94651B0C94DA
:10232000A31B9BE5980F933020F480E090E00C9481
:10233000750F885A853120F480E090E00C94A30F4B
:102340000895882321F00E945F1B0C94A31B08951D
:10235000882321F00E94651B0C94A31B0895BF9253
:10236000CF92DF92EF92FF920F931F93CF93DF9361
:1023700000D000D000D0CDB7DEB725E0FC01DE01F3
:10238000119601900D922A95E1F7FC01408151814F
:10239000028163817481258122952F7061157105F9
:1023A00009F403C35F3F19F44F3F09F4FEC26C0107
:1023B000862F7D836C83602F782F8D812E830E94E2
:1023C000381A182FB92E0E94371A0E942719EB2DA0
:1023D000E295EF70F0E0E05AFF4F2E810C946625F5
:1023E0008B2D807F9B2D9F70F92E882319F0F294FE
:1023F00090EFF922002349F0FF2009F483C28F2DCA
:102400000E94721B0E94A31B7DC2812F0E94751126
:10241000FF2009F4CAC28F2D0E94781B26960FB6A2
:10242000F894DEBF0FBECDBFDF91CF911F910F910A
:10243000FF90EF90DF90CF90BF900C94A31B8B2D5B
:10244000807F9B2D9F70F92E803219F0F29480EFDF
:10245000F822112319F0113009F12AC00023B1F03C
:102460008F2D222351F1213041F526960FB6F89495
:10247000DEBF0FBECDBFDF91CF911F910F91FF90B7
:10248000EF90DF90CF90BF900C94821B222319F025
:10249000213009F48AC20E948B1B2DC00023F1F069
:1024A000263008F082C20E945C1B8F2129F023C0D5
:1024B0000023F9F0211116C08F2D26960FB6F8943F
:1024C000DEBF0FBECDBFDF91CF911F910F91FF9067
:1024D000EF90DF90CF90BF900C94A111253008F0C1
:1024E00064C209C0F601858180FF0CC28F708583AC
:1024F000E3CF21111CC28F2D83C12B2D269526954C
:10250000237030E02115310521F021303105D1F063
:102510004CC2002321F0812F9B2D937002C080E0DC
:1025200090E026960FB6F894DEBF0FBECDBFDF91C8
:10253000CF911F910F91FF90EF90DF90CF90BF90C0
:102540000C94750F002321F0812F9B2D937002C0F6
:1025500080E090E026960FB6F894DEBF0FBECDBFA8
:10256000DF91CF911F910F91FF90EF90DF90CF906F
:10257000BF900C94A30F812F002319F00E94FC1D23
:1025800002C00E94641E26960FB6F894DEBF0FBEEE
:10259000CDBFDF91CF911F910F91FF90EF90DF9012
:1025A000CF90BF900C94E91E8B2D837009F07BC0F7
:1025B0000111FBC1812F829586958770880F880F46
:1025C000912F9F70C92ED12CE12CF12C082E04C024
:1025D000CC0CDD1CEE1CFF1C0A94D2F714FF12C0B9
:1025E0004FE050E060E070E004C0440F551F661FEC
:1025F000771F8A95D2F7CB01BA01609570958095C7
:10260000909503C060E070E0CB012B2D26952695B8
:102610002370422F50E042305105D9F0433051052C
:1026200069F16C297D298E299F294130510551F18D
:1026300026960FB6F894DEBF0FBECDBFDF91CF91C7
:102640001F910F91FF90EF90DF90CF90BF900C946F
:102650004C196C297D298E299F2926960FB6F8944E
:10266000DEBF0FBECDBFDF91CF911F910F91FF90C5
:10267000EF90DF90CF90BF900C9466190E944C1998
:10268000C701B60126960FB6F894DEBF0FBECDBFC8
:10269000DF91CF911F910F91FF90EF90DF90CF903E
:1026A000BF900C943219002319F08B2D817001C05A
:1026B0008695882309F479C1812F82958695877044
:1026C000880F880F912F9F70C92ED12CE12CF12CEF
:1026D000082E04C0CC0CDD1CEE1CFF1C0A94D2F7A3
:1026E00014FF12C04FE050E060E070E004C0440FFF
:1026F000551F661F771F8A95D2F7CB01BA016095E7
:1027000070958095909503C060E070E0CB012B2D13
:10271000269526952370422F50E042305105D9F07E
:102720004330510569F16C297D298E299F2941305B
:10273000510551F126960FB6F894DEBF0FBECDBFFE
:10274000DF91CF911F910F91FF90EF90DF90CF908D
:10275000BF900C94131A6C297D298E299F292696E7
:102760000FB6F894DEBF0FBECDBFDF91CF911F91A2
:102770000F91FF90EF90DF90CF90BF900C94251AAF
:102780000E94131AC701B60126960FB6F894DEBF51
:102790000FBECDBFDF91CF911F910F91FF90EF90B2
:1027A000DF90CF90BF900C94011A103FD1F128F424
:1027B00080E4810F803250F0A0C0123F09F462C063
:1027C00008F44BC0133F09F472C097C0F12FF071A9
:1027D000FF2E8B2D8F71002351F00E949A19812FAB
:1027E000FF2019F08295807F68CE8F7066CE0E94A0
:1027F000BB19812FFF2019F08295807F01C08F7057
:1028000026960FB6F894DEBF0FBECDBFDF91CF91F5
:102810001F910F91FF90EF90DF90CF90BF900C949D
:10282000A8110023B1F0253008F0BFC08B2D8F71A7
:1028300026960FB6F894DEBF0FBECDBFDF91CF91C5
:102840001F910F91FF90EF90DF90CF90BF900C946D
:10285000E019263008F0A9C0E9CF0023A9F08B2D9C
:102860008F7126960FB6F894DEBF0FBECDBFDF91F5
:10287000CF911F910F91FF90EF90DF90CF90BF907D
:102880000C949A19002359F38B2D8F7126960FB64D
:10289000F894DEBF0FBECDBFDF91CF911F910F9196
:1028A000FF90EF90DF90CF90BF900C94BB19002366
:1028B00099F08B2D8F7126960FB6F894DEBF0FBE60
:1028C000CDBFDF91CF911F910F91FF90EF90DF90DF
:1028D000CF90BF900C94851926960FB6F894DEBF62
:1028E0000FBECDBFDF91CF911F910F91FF90EF9061
:1028F000DF90CF90BF900C9480190023A9F0222381
:1029000009F4ADCF812F26960FB6F894DEBF0FBE27
:10291000CDBFDF91CF911F910F91FF90EF90DF908E
:10292000CF90BF900C940A11222309F4ADCF812FD0
:1029300026960FB6F894DEBF0FBECDBFDF91CF91C4
:102940001F910F91FF90EF90DF90CF90BF900C946C
:1029500075114B2D4F70612FC6010E94761D269672
:102960000FB6F894DEBF0FBECDBFDF91CF911F91A0
:102970000F91FF90EF90DF90CF90BF900C94801854
:102980004B2D4F70612FC60126960FB6F894DEBF0F
:102990000FBECDBFDF91CF911F910F91FF90EF90B0
:1029A000DF90CF90BF900C94791D26960FB6F894C7
:1029B000DEBF0FBECDBFDF91CF911F910F91FF9072
:1029C000EF90DF90CF90BF9008950E947F1B0E94F0
:1029D0004E1B0E94A31B0E941B200E94E91E80E048
:1029E00090E00E94750F80E090E00C94A30F0E948D
:1029F0006F1B0C94E514CF93DF9300D000D01F928F
:102A0000CDB7DEB7942F4983252F5A836B837C8300
:102A10008D834C815D81452B39F12F3F11F49F3F10
:102A200019F149815A816B817C818D810E94381A0C
:102A3000292F22952F7030E02C30310504F52A30F3
:102A400031055CF4225031092230310568F4853AB1
:102A500080F4843090F4823080F0883E38F4803EF8
:102A600060F48450813A48F080E014C0803FE1F780
:102A700004C090E2980F983080F781E00BC02C30B2
:102A8000310521F493FB882780F904C02F303105EC
:102A9000C9F3EACF0F900F900F900F900F90DF9136
:102AA000CF910895CF93DF9300D000D01F92CDB780
:102AB000DEB70F900F900F900F900F90DF91CF9196
:102AC0000895CF93DF9300D000D000D0CDB7DEB70C
:102AD00026960FB6F894DEBF0FBECDBFDF91CF9123
:102AE00008951F93CF93DF93C0919F0116E08091CB
:102AF000A001C81799F0D0E01C9FF0011D9FF00DB8
:102B00001124EF55FE4F4081518162817381848190
:102B100095810E9461152196C770E9CFDF91CF9111
:102B20001F9108954091D1015091D2016091D3013C
:102B30007091D4018091D5019091D6010C946115CA
:102B40008091D60182958F7009F054C08091D30195
:102B5000882309F44FC080919F01A091A00160914A
:102B6000D1017091D2014091D4015091D501B6E0CC
:102B70008A1709F43FC090E041155105C1F17F3F2C
:102B800011F46F3FA1F1B89FF001B99FF00D11242E
:102B9000EF55FE4F218172132AC02081621327C096
:102BA0002281211124C0238134812417350710F498
:102BB00021503109241B350B2C323140C0F42091B7
:102BC000D6012F7020612093D60126E0289FF001C6
:102BD000299FF00D1124EA55FE4F80818F7080618E
:102BE000808381ED91E00E94AF110C9471150196E4
:102BF0008770BECF0895BF92CF92DF92EF92FF927F
:102C00000F931F93CF93DF93CDB7DEB761970FB6C6
:102C1000F894DEBF0FBECDBF7C0185E0F701DE0179
:102C20001D9601900D928A95E1F7D7014C9111966E
:102C30005C9111971296DC90129713960D911C914E
:102C400014973091D1016091D2018091D40190917B
:102C5000D501009709F47FC16F3F19F43F3F09F494
:102C60007AC1B090D301BB2009F4CAC02091D6012B
:102C70000817190750F0F801E81BF90BCF01CC2415
:102C8000C3948C329140D0F009C080959095800F0C
:102C9000911FCC24C3948C32914080F0C12C207FB2
:102CA00009F0CCC0702F198B088B6D2D89890E947B
:102CB000521581ED91E00E94AF11B6C0822F807F46
:102CC00009F047C0651314C0341312C0D11010C0EE
:102CD0002F7020612093D6010E94921581ED91E022
:102CE0000E94AF118091D601D70115968C932FC009
:102CF0000115110519F15F3F11F44F3FF9F0CD2C8B
:102D0000D1101CC080919F012091A00136E0821754
:102D100009F45CC090E0389FF001399FF00D112458
:102D2000EF55FE4F6181561306C06081461303C004
:102D30006281611103C001968770E9CFCD2CDD203F
:102D400009F429C18091D60181608093D601C12CFC
:102D500022C1651308C0341306C0D11004C080918D
:102D6000D601D701CCC04D875E87DF86702F198BC7
:102D7000088B6D2D89890E94FB148823E9F1DD20E1
:102D8000D9F12091D601822F82958F7090E0029721
:102D900074F08091D1019091D20198878F83198628
:102DA0001B870A872C87CE0107960E94AF1186E009
:102DB000F701A1EDB1E001900D928A95E1F70E9433
:102DC000A0150E949215CC24C394E5C0702F198BD6
:102DD000088B60E089890E94381A292F22952F706C
:102DE00030E0223031050CF0CAC09F7009F0C4C039
:102DF000805E883008F4CFC0C7010E94AF11E3CFD6
:102E00000817190708F456C0F801E81BF90BCF01A1
:102E10008C32914008F456C0C12C702F198B088B4E
:102E20006D2D89890E945215E1EDF1E086E0DF0108
:102E30001D928A95E9F70E949215ADC0651314C0E2
:102E4000341312C0D11010C08091D601F7018583D0
:102E5000C7010E94AF1186E0E1EDF1E0DF011D92B4
:102E60008A95E9F7CB2C97C04D875E87DF86702F58
:102E7000198B088B6D2D89890E94FB14882309F416
:102E8000BBCFDD2009F4B8CF2091D601822F8295E7
:102E90008F7090E002970CF48ACF8091D1019091CD
:102EA000D2019A8389831B821D830C832E83CE01DA
:102EB00001967BCF80959095800F911F8C32914029
:102EC00008F0AACFCD2CDD2009F496CF65132EC0D3
:102ED00034132CC02091D60120FD1FC0822F829573
:102EE0008F70D9F0D70115962C9315978F3049F034
:102EF0008F5F982F9295907F822F8F70892B1596D8
:102F00008C93C7010E94AF1186E0F701A1EDB1E0FB
:102F100001900D928A95E1F78ECF86E0F701A1ED41
:102F2000B1E001900D928A95E1F735C04D875E873B
:102F3000DF86702F198B088B6D2D89890E94FB14F9
:102F4000811135CF8091D60181608093D601C70170
:102F50000E94AF1120C0DD2009F44ECF4D875E875F
:102F6000DF86702F198B088B6D2D89890E94FB14C9
:102F7000882309F441CF1BCF81113ACF0CC02430F4
:102F800031050CF039CF9F7009F432CFF7019581EC
:102F9000907F09F02DCF8C2D61960FB6F894DEBF8F
:102FA0000FBECDBFDF91CF911F910F91FF90EF909A
:102FB000DF90CF90BF9008951F93CF93DF93CDB74D
:102FC000DEB72C970FB6F894DEBF0FBECDBF4F8390
:102FD000588769877A878B879C87CE0107960E94DE
:102FE000FB15882369F08F8198852A853B85232BE3
:102FF000F1F19F3F09F063C08F3F09F060C037C017
:1030000086E0FE013796DE01119601900D928A95B9
:10301000E1F76F817885EA85FB85309741F17F3F45
:1030200011F46F3F21F12091A00130E0C901019618
:103030008770992740919F0150E08417950709F404
:1030400047C069837A83FD83EC8396E0929FD00129
:10305000939FB00D1124AF55BE4FFE0131960190E4
:103060000D929A95E1F78093A0010E94711516E0E8
:1030700080919F019091A0018917C1F1189FC00113
:1030800011248F559E4F0E94FB15882379F1E09102
:103090009F011E9FF0011124EF55FE4F4081518189
:1030A00062817381848195810E94611580919F0165
:1030B00090E001968770992780939F01D9CF4F8127
:1030C000588569857A858B859C850E946115CFCF4F
:1030D0000E94F7141092A00110929F01E1EDF1E01F
:1030E00086E0DF011D928A95E9F7C1CF2C960FB6D5
:1030F000F894DEBF0FBECDBFDF91CF911F91089531
:10310000DF92EF92FF920F931F93CF93DF93FC0117
:10311000892B09F48AC0E12CF12CDD24D394EF0132
:1031200021968491853709F461C058F4843708F0FA
:103130004EC0843008F06AC08130D1F0823071F125
:1031400074C0883709F45DC050F4863709F455C05F
:10315000873709F06AC08E2D0E946C1B54C09CE713
:10316000980F903708F061C08F770E94751150C09A
:103170008F010E5F1F4FFE01849190E2980F9830EF
:1031800050F48770FD2D01C0FF0F8A95EAF78F2F4D
:103190000E94721B14C00E940A1113C08F010E5F9F
:1031A0001F4FFE01C49180E28C0F883060F4C7701D
:1031B0008D2D01C0880FCA95EAF70E94781B0E94E6
:1031C000A31BE80125C08C2F0E947511FACF9F0127
:1031D0002E5F3F4FFE01C491CC2369F08FE99FE041
:1031E0000197F1F700C00000C150F6CF9F012E5F9C
:1031F0003F4FFE01F490E9010BC00E945C1BE82EDA
:1032000007C00E946F1B0E94A31B02C00E940A11EC
:103210008F2D882341F0EFE9FFE03197F1F700C0EF
:1032200000008150F6CFFE017ACFDF91CF911F9140
:103230000F91FF90EF90DF90089560935702709385
:1032400058028093590290935A020C943E1C0895A0
:1032500060935B0270935C0280935D0290935E02C8
:103260000C943D1C0F931F9300915B0210915C0224
:1032700020915D0230915E02602B712B822B932B8B
:1032800060935B0270935C0280935D0290935E0298
:103290001F910F910C943D1C0F931F9300915B02A3
:1032A00010915C0220915D0230915E0260237123D7
:1032B0008223932360935B0270935C0280935D0290
:1032C00090935E021F910F910C943D1C0F931F93DE
:1032D00000915B0210915C0220915D0230915E02D0
:1032E000602771278227932760935B0270935C02AB
:1032F00080935D0290935E021F910F910C943D1C90
:1033000060E070E0CB010C941D190F931F9341E016
:1033100050E060E070E08A019B0104C0000F111FC3
:10332000221F331F8A95D2F7C901B8011F910F914F
:103330000C941D190F931F9341E050E060E070E082
:1033400004C0440F551F661F771F8A95D2F78091DE
:10335000570290915802A0915902B0915A028A01E5
:103360009B01082B192B2A2B3B2BC901B8011F915C
:103370000F910C941D190F931F9341E050E060E0F2
:1033800070E004C0440F551F661F771F8A95D2F75F
:103390004095509560957095809157029091580294
:1033A000A0915902B0915A028A019B010823192366
:1033B0002A233B23C901B8011F910F910C941D19B9
:1033C0000F931F9341E050E060E070E004C0440FB1
:1033D000551F661F771F8A95D2F7809157029091EB
:1033E0005802A0915902B0915A028A019B01082704
:1033F00019272A273B27C901B8011F910F910C9467
:103400001D190F931F93009157021091580220919C
:10341000590230915A02602B712B822B932B1F91F2
:103420000F910C941D190F931F9300915702109147
:1034300058022091590230915A026023712382234D
:1034400093231F910F910C941D190F931F930091BB
:103450005702109158022091590230915A02602768
:103460007127822793271F910F910C941D1908959E
:103470008F929F92AF92BF92DF92EF92FF920F9343
:103480001F93CF93DF9300D000D01F92CDB7DEB74C
:103490006B837C838D838A018C819D81892B21F0B4
:1034A0001F3F29F44F3F19F480E090E04CC08B811E
:1034B0008823C9F180905B0290905C02A0905D022D
:1034C000B0905E028091570290915802A0915902EB
:1034D000B0915A02882A992AAA2ABB2A8FE1E82E9B
:1034E000F12CD501C4010E2C04C0B695A795979573
:1034F00087950A94D2F780FF07C0DE2CB8018E2D85
:103500000E944C1D019729F481E0E81AF10848F760
:10351000D12C80E1189FF0011124E00FF11DE95238
:10352000FE4FD08209C080E1189FF0011124E00F06
:10353000F11DE952FE4FD08009831A8369817A8197
:103540008D2D0E944C1D0F900F900F900F900F909B
:10355000DF91CF911F910F91FF90EF90DF90BF907F
:10356000AF909F908F90089590910A01992321F038
:1035700090910B01911109C020910C0130910D0126
:10358000F90132969FEF40E030C0982F96959695BE
:1035900096959F31A0F4E0910C01F0910D01E90F97
:1035A000F11D877021E030E0A90102C0440F551FD2
:1035B0008A95E2F7CA019181892B818308959091C0
:1035C000840290FF23C01F928F938CE094E09F931E
:1035D0008F930E942E060F900F900F900F900895DA
:1035E0009F3F39F04F5F4E3141F051915813F8CF62
:1035F0000DC05111F7CF942FF5CF9F3F39F0F9014E
:10360000E90FF11D97FDFA95828308950895909131
:103610000A01992321F090910B01911109C0209189
:103620000C0130910D01F9013296205E3F4F30C000
:10363000982F9695969596959F31A8F4E0910C0158
:10364000F0910D01E90FF11D877021E030E0A90133
:1036500002C0440F551F8A95E2F7CA0180959181F7
:103660008923818308959091840290FF16C01F9250
:103670008F938EEE93E09F938F930E942E060F9070
:103680000F900F900F9008953196E217F30729F0ED
:1036900090819813F9CF1082F7CF089581E090E0E0
:1036A000E0910C01F0910D01E80FF91F10820196D5
:1036B00080329105A9F70895809183020895909131
:1036C0008302892B809383020895809590918302D1
:1036D0008923809383020895809383020895109232
:1036E0008302089590918202892B8093820208952B
:1036F000809590918202892380938202089510928E
:1037000082020895809361020E94B51C909360022A
:1037100080935F02089510926102109260021092ED
:103720005F02089580910C0190910D01FC0131968A
:103730009C01205E3F4F80E0919191118F5FE217D5
:10374000F307D1F70895E0910C01F0910D018091FC
:1037500083028083E0910C01F0910D0190818091B2
:103760008202892B8083809161028823D9F10E9493
:10377000B51C20915F02309160028217930748F0D8
:103780000E94B51C20915F0230916002821B930B56
:103790000AC00E94B51C20915F0230916002209502
:1037A0003095820F931F8C32914070F0809184028B
:1037B00080FF08C08AE294E09F938F930E942E06B8
:1037C0000F900F900E948B1BE0910C01F0910D0166
:1037D000908180916102892B80830E94921B8111CC
:1037E0000E948B1B80910C0190910D010C94210F74
:1037F000909339018093380108958295982F9C7C8D
:10380000392F36953695282F237344E0249FC00125
:103810001124932F982B292F2A7A2695892F857585
:10382000880F822B08951F93CF93DF931F92CDB7FC
:10383000DEB799830E94FD1B182F9981892F0E9462
:10384000FD1B212F30E0322F2227A901482BCA016E
:103850000F90DF91CF911F9108950895CF93DF933B
:1038600000D000D01F92CDB7DEB70F900F900F9011
:103870000F900F90DF91CF910895089508950C94C3
:10388000901080919902843021F11092850220E4F9
:1038900088E190E00FB6F894A895809360000FBE81
:1038A0002093600083B7817F846083BF83B781608A
:1038B00083BF7894889583B78E7F83BF0FB6F894C3
:1038C000A8958091600088618093600010926000EC
:1038D0000FBE0895CF930E94C8100E9465060E94F3
:1038E000C910C0E08C2F0E942907892B29F4CF5FD3
:1038F000C830C1F780E001C081E0CF9108950E94F7
:1039000092100C94F7141F920F920FB60F9211247D
:103910008F939F93AF93BF9380918502811113C0C2
:103920008091860290918702A0918802B0918902CD
:103930004196A11DB11D8093860290938702A093AA
:103940008802B0938902BF91AF919F918F910F90A0
:103950000FBE0F901F90189582E084BD93E095BD37
:103960009AEF97BD80936E0008952FB7F8948091D9
:10397000860290918702A0918802B09189022FBFA0
:1039800008952FB7F8946091860270918702809114
:103990008802909189022FBF0895CF92DF92EF9213
:1039A000FF920F931F932FB7F89440918602509186
:1039B000870260918802709189022FBF6A017B01A2
:1039C000EE24FF248C0120E030E0C016D106E20690
:1039D000F30610F4415051099A01281B390BC90113
:1039E0001F910F91FF90EF90DF90CF9008951F925D
:1039F0000F920FB60F9211248F939F93AF93BF93A3
:103A00008091860290918702A0918802B0918902EC
:103A10000196A11DB11D8093860290938702A09309
:103A20008802B0938902BF91AF919F918F910F90BF
:103A30000FBE0F901F9018950E942E0CF8942FEF38
:103A400087EA91E6215080409040E1F700C00000F5
:103A500087E090EBDC018093A2029093A302A093F5
:103A6000A402B093A5029CE088E10FB6F894A89553
:103A7000809360000FBE90936000FFCF20E1929F83
:103A8000F0011124E80FF11DE052FF4F9491892FAE
:103A90008F7092959F700895CF93C82FCB010E948D
:103AA0003E1D282F30E080E1989FA0011124422B79
:103AB000532B4038510519F480E090E015C0977001
:103AC000E92FF0E088E0C89FE00DF11D112484E0AB
:103AD000EE0FFF1F8A95E1F7E20FF31FEE0FFF1FB6
:103AE000E050F84985919491CF91089580E090E05D
:103AF0000895089580918C0280FF0BC060911101A0
:103B000085E0689FB0011124759567957595679557
:103B10002BC081FF09C06091110185E0689FB00151
:103B200011247595679520C082FF07C0609111012F
:103B300085E0689FB001112417C090918D029923F0
:103B4000D1F060911001961788F72091110185E05E
:103B5000289F90011124929FA001939F500D112442
:103B600070E0CA010E9452256038710540F4611569
:103B7000710539F002C065E070E0862F08958FE787
:103B8000089581E0089580918C0280FF08C06091C3
:103B90000F0170E0759567957595679521C081FF58
:103BA00006C060910F0170E07595679519C082FF9E
:103BB00004C060910F0170E010C090918D029923B4
:103BC000C1F060910E019617A0F780910F01899FB7
:103BD000C001112470E00E9452256038710528F45C
:103BE0006115710521F0862F08958FE7089581E012
:103BF000089561E070E0F4CF803F21F40E947A1DC7
:103C0000819504C0813F29F40E947A1D809390021F
:103C10000895823F21F40E947A1D819504C0833F5C
:103C200029F40E947A1D80938F020895893F19F428
:103C30000E94C31D05C08A3F31F40E94C31D8195B7
:103C40008093910208958B3F21F40E94C31D8195BA
:103C500004C08C3F29F40E94C31D809392020895F2
:103C6000843F21F480918E02816017C0853F21F44A
:103C700080918E02826011C0863F21F480918E0275
:103C800084600BC0873F21F480918E02886005C05C
:103C9000883F31F480918E02806180938E02089576
:103CA0008D3F21F480918C0281600BC08E3F21F406
:103CB00080918C02826005C08F3F29F480918C0234
:103CC000846080938C020895803F39F48091900243
:103CD00087FF6CC01092900269C0813F29F48091E7
:103CE00090021816BCF362C090918F02823F29F4B3
:103CF00097FF5CC010928F0259C0833F19F41916C8
:103D0000CCF354C0893F41F48091910218160CF015
:103D10004DC0109291024AC08A3F29F480919102CD
:103D200087FF44C0F6CF8B3F39F48091920287FF22
:103D30003DC0109292023AC08C3F29F480919202C9
:103D40001816BCF333C0843F21F480918E028E7F1D
:103D500017C0853F21F480918E028D7F11C0863F70
:103D600021F480918E028B7F0BC0873F21F48091DC
:103D70008E02877F05C0883F31F480918E028F7E4E
:103D800080938E0213C08D3F21F480918C028E7F30
:103D90000BC08E3F21F480918C028D7F05C08F3F38
:103DA00029F480918C028B7F80938C0280918F020A
:103DB00081110EC08091900281110AC08091910200
:103DC000811106C080919202811102C010928D0271
:103DD00008958091840283FF7EC083E694E00E9470
:103DE000950580918E021F928F938EE594E09F93AC
:103DF0008F930E942E068CE594E00E949505809199
:103E00008F02282F082E000C330B3F938F9389E5E8
:103E100094E09F938F930E942E0687E594E00E9482
:103E2000950580919002282F082E000C330B3F93AC
:103E30008F9384E594E09F938F930E942E0682E5F2
:103E400094E00E94950580919102282F082E000C85
:103E5000330B3F938F938FE494E09F938F930E9453
:103E60002E068DE494E00E94950580919202282F01
:103E7000082E000C330B3F938F938AE494E09F93BA
:103E80008F930E942E0687E494E00E94950580910E
:103E90008D021F928F9384E494E09F938F930E94EE
:103EA0002E0682E494E00E94950580918C021F9278
:103EB0008F938FE394E09F938F930E942E068CE361
:103EC00094E00E9495058DB79EB74C960FB6F89476
:103ED0009EBF0FBE8DBF8EE892E00E946A0F0E94C7
:103EE000B51C90938B0280938A0208951F93CF9301
:103EF000DF9380918A0290918B020E94CD1CAC01CD
:103F000090918D02992321F02091120130E006C09A
:103F1000209113018AE0289F900111244217530732
:103F200008F485C080918F02C0919002D0919102D7
:103F300010919202811107C0C11175C0D11173C0D7
:103F4000111171C074C09F3F19F09F5F90938D0253
:103F5000181624F40E947A1D80938F0280918F029C
:103F600087FF05C00E947A1D819580938F021C16E1
:103F700024F40E947A1D809390028091900287FF22
:103F800005C00E947A1D81958093900260918F02F6
:103F9000662331F1C0919002CC2311F1062E000C62
:103FA000770B880B990B0E944D2423E333E343E303
:103FB0005FE30E94B1240E94152460938F026C2F4E
:103FC000CC0F770B880B990B0E944D2423E333E32E
:103FD00043E35FE30E94B1240E94152460939002A2
:103FE0001D1624F40E94C31D8093910280919102BA
:103FF00087FF05C00E94C31D819580939102111611
:1040000024F40E94C31D809392028091920287FF44
:1040100005C00E94C31D819580939202DF91CF91CC
:104020001F910C94E91E9F3F09F08FCF97CFDF912E
:10403000CF911F910895EEE8F2E085E0DF011D9237
:104040008A95E9F710928D0210928C02089586E805
:1040500096E00E9495051F9281E08F931F9285E064
:104060008F9388E396E09F938F930E942E060F9084
:104070000F900F900F900F900F9008958330E9F1FB
:1040800028F4813061F0823009F10895853009F417
:1040900062C008F449C0863009F474C00895809164
:1040A0001301262F30E0280F311D2F3F310524F456
:1040B000680F6093130103C08FEF80931301809109
:1040C00013011F928F9381E795E072C080911201D6
:1040D000262F30E0280F311D2F3F310524F4680FC3
:1040E0006093120103C08FEF80931201809112013F
:1040F0001F928F938FE595E05BC080911101262F71
:1041000030E0280F311D2F3F310524F4680F6093F4
:10411000110103C08FEF80931101809111011F9253
:104120008F938CE495E044C080911001262F30E0FD
:10413000280F311D2F3F310524F4680F60931001C3
:1041400003C08FEF80931001809110011F928F9315
:1041500087E395E02DC080910F01262F30E0280FD6
:10416000311D2F3F310524F4680F60930F0103C008
:104170008FEF80930F0180910F011F928F938EE13B
:1041800095E016C080910E01262F30E0280F311DDA
:104190002F3F310524F4680F60930E0103C08FEFA9
:1041A00080930E0180910E011F928F9383E095E022
:1041B0009F938F930E942E060F900F900F900F9059
:1041C0000895833081F128F4813059F08230D1F0A4
:1041D0000895853009F449C0B8F1863009F456C015
:1041E000089580911301681720F4861B80931301B2
:1041F00002C010921301809113011F928F9384EFDC
:1042000094E054C080911201681720F4861B8093BB
:10421000120102C010921201809112011F928F931D
:1042200082EE94E043C080911101681720F4861B50
:104230008093110102C010921101809111011F920F
:104240008F938FEC94E032C080911001681720F4B6
:10425000861B8093100102C0109210018091100102
:104260001F928F938AEB94E021C080910F01681711
:1042700020F4861B80930F0102C010920F018091E1
:104280000F011F928F9381EA94E010C080910E017C
:10429000681720F4861B80930E0102C010920E0155
:1042A00080910E011F928F9386E894E09F938F93E5
:1042B0000E942E060F900F900F900F900895CF93AD
:1042C000C82F1F928F938BE897E09F938F930E9444
:1042D0002E0681E090E0A0E0B0E0BC01CD0104C07A
:1042E000660F771F881F991FCA95D2F70E94281959
:1042F0000F900F900F900F90CF910C94F714CF93D5
:104300008732A8F58E3108F02BC1803109F49FC0A7
:10431000F8F4873009F464C0A8F4863009F024C1A9
:1043200080918402817F8E7F8093840280E997E070
:104330000E9495058BE79AE00E94950581E08093A5
:1043400094024CC08B30F1F18E3009F46CC00CC17A
:10435000863109F4B0C020F4813109F4EDC004C104
:10436000893109F491C08B3109F449C0FDC088330B
:1043700049F150F4893209F4F1C0853309F4EEC0F3
:10438000873209F0F1C0EAC0833409F4E7C028F4A9
:104390008A3308F4E9C08953E4C0883409F0E4C0E2
:1043A0000E94F7148AE69AE00E9495052FEF83EDAC
:1043B00090E3215080409040E1F700C000000E944F
:1043C0001C1D0CC087EB97E05CC081E59AE00E9461
:1043D000950580918402816080938402C1E0C9C008
:1043E00080918402C82FC17080FFEFCF8DE59AE0E5
:1043F0000E94950580918402817F8E7F3DC09091BF
:10440000840291FBCC27C0F981E0C827892FC0FB2B
:1044100081F980938402CC2319F084E49AE027C0C8
:1044200086E39AE02EC09091840292FBCC27C0F9DB
:1044300081E0C827892FC0FB82F980938402CC23B6
:1044400019F087E29AE013C087E19AE01AC09091D0
:10445000840293FBCC27C0F981E0C827892FC0FBD9
:1044600083F980938402CC2351F08BE09AE00E9480
:104470009505809184028160809384027AC08EEFDA
:1044800099E00E949505AACF8FEE99E00E949505CC
:1044900086EC99E00E94950584E899E00E949505D4
:1044A0008DE599E00E94950583E199E00E949505CC
:1044B00085EE98E0E6CF87ED98E00E9495050E9492
:1044C000150F1F928F938DEB98E09F938F930E940F
:1044D0002E0680910A011F928F9386EA98E09F939F
:1044E0008F930E942E06809187011F928F9383E9FC
:1044F00098E09F938F930E942E0680910B011F924C
:104500008F9380E898E09F938F930E942E060E94DD
:10451000C11C9F938F937F936F9389E698E09F933D
:104520008F930E942E068DB79EB746960FB6F894CD
:104530009EBF0FBE8DBF52CF0E94F714C0910B01DA
:1045400081E0C827C0930B01CC2329F08FE598E0C8
:104550000E9495050EC084E598E093CF80E001C0ED
:104560008D510E945F213ACF82E598E00E94950527
:10457000C0E08C2FCF91089580E0089580E00895E9
:10458000CF93C82F80919402813071F020F0823057
:1045900009F44BC042C1E0910C01F0910D01808102
:1045A000823209F03CC107C0E0910C01F0910D018D
:1045B0008081823261F48C2F0E94BC22811104C060
:1045C0008C2F0E947F212FC081E090E02CC08C2F87
:1045D0000E94BE22811126C0C431E1F070F4CB30BC
:1045E00081F0C031D1F40E94272083E897E00E9437
:1045F000950582E08093940215C0C93259F0C83302
:1046000061F480E997E00E94950587E897E00E94B1
:10461000950508C01092940204C181E897E00E94B9
:104620009505FFC081E08170FEC0C43228F5CE310F
:1046300008F0C1C0CB30A1F1D0F4C73009F0D3C02D
:104640008EE18093130182E3809312018AE08093CC
:10465000110184E18093100188E080930F0188E2CA
:1046600080930E0187E296E00E949505BFC0C3319A
:1046700049F1C431C1F0B7C0CB3409F4A9C028F462
:10468000C93289F0C83361F0AEC0C13509F49EC0AB
:10469000C23509F499C0CE3409F0A5C06AE09EC0C5
:1046A0000E942720A3C080919302882319F01092C2
:1046B00093029CC084E396E00E94950581E080937C
:1046C0009402B1C08EE096E00E9495058CEF95E0D3
:1046D0000E949505809113011F928F9389EF95E0B9
:1046E0009F938F930E942E0687EF95E00E94950579
:1046F00085EE95E00E949505809112011F928F939F
:1047000082EE95E09F938F930E942E0680EE95E0B7
:104710000E94950581ED95E00E949505809111011B
:104720001F928F938EEC95E09F938F930E942E069D
:104730008CEC95E00E9495058BEB95E00E94950529
:10474000809110011F928F9388EB95E09F938F9338
:104750000E942E0686EB95E00E94950581EA95E081
:104760000E94950580910F011F928F938EE995E02D
:104770009F938F930E942E068CE995E00E949505E9
:1047800085E895E00E94950580910E011F928F9318
:1047900082E895E09F938F930E942E0680E895E033
:1047A0000E9495058DB79EB748960FB6F8949EBFA8
:1047B0000FBE8DBF1BC0CE51EC2FF0E0E25DFE4F6F
:1047C00080818093930212C061E003C061E006C063
:1047D0006AE0809193020E943E2008C0809193027B
:1047E0000E94E12003C085E296E013C0809193020D
:1047F000882369F01F928F938FE196E09F938F93A8
:104800000E942E060F900F900F900F9004C08CE125
:1048100096E00E94950581E006C01092940280E027
:1048200002C080E000CFCF9108950E941C246894BC
:10483000B1110C94AB2408950E94902488F09F57E6
:1048400098F0B92F9927B751B0F0E1F0660F771FB4
:10485000881F991F1AF0BA95C9F714C0B13091F0AA
:104860000E94AA24B1E008950C94AA24672F782FFF
:104870008827B85F39F0B93FCCF38695779567956F
:10488000B395D9F73EF490958095709561957F4FDB
:104890008F4F9F4F0895E89409C097FB3EF4909581
:1048A0008095709561957F4F8F4F9F4F9923A9F009
:1048B000F92F96E9BB279395F69587957795679598
:1048C000B795F111F8CFFAF4BB0F11F460FF1BC0DC
:1048D0006F5F7F4F8F4F9F4F16C0882311F096E96F
:1048E00011C0772321F09EE8872F762F05C066231D
:1048F00071F096E8862F70E060E02AF09A95660FD6
:10490000771F881FDAF7880F9695879597F908958E
:1049100057FD9058440F551F59F05F3F71F0479570
:10492000880F97FB991F61F09F3F79F08795089555
:10493000121613061406551FF2CF4695F1DF08C074
:10494000161617061806991FF1CF86957105610591
:1049500008940895E894BB2766277727CB0197F939
:1049600008950E94C4240C9435250E94272538F010
:104970000E942E2520F0952311F00C941E250C94F6
:10498000242511240C94AB240E94882470F3959F55
:10499000C1F3950F50E0551F629FF001729FBB2736
:1049A000F00DB11D639FAA27F00DB11DAA1F649FD2
:1049B0006627B00DA11D661F829F2227B00DA11D85
:1049C000621F739FB00DA11D621F839FA00D611D0B
:1049D000221F749F3327A00D611D231F849F600D2C
:1049E000211D822F762F6A2F11249F5750409AF055
:1049F000F1F088234AF0EE0FFF1FBB1F661F771FE1
:104A0000881F91505040A9F79E3F510580F00C94AB
:104A10001E250C94AB245F3FE4F3983ED4F38695B7
:104A200077956795B795F795E7959F5FC1F7FE2B4B
:104A3000880F911D9695879597F9089597F99F6727
:104A400080E870E060E008959FEF80EC0895002416
:104A50000A941616170618060906089500240A94E3
:104A600012161306140605060895092E0394000C69
:104A700011F4882352F0BB0F40F4BF2B11F460FFF8
:104A800004C06F5F7F4F8F4F9F4F0895991B79E050
:104A900004C0991F961708F0961B881F7A95C9F7CE
:104AA0008095089597FB072E16F4009407D077FDA4
:104AB00009D00E946C2507FC05D03EF490958195A5
:104AC0009F4F0895709561957F4F0895EE0FFF1FDA
:104AD0000590F491E02D0994AA1BBB1B51E107C07E
:104AE000AA1FBB1FA617B70710F0A61BB70B881F7E
:104AF000991F5A95A9F780959095BC01CD0108950D
:044B0000F894FFCF57
:104B0400460737081408E007AC07010162022808C9
:104B1400140A321E404D3622394D030003CA02A83E
:104B2400026F02E201FB0114022D024D0200010298
:084B340003040506070809004F
:106800000000000000000000040005000600070072
:10681000080009000A000B000C000D000E000F001C
:1068200010001100120013001400150016001700CC
:10683000180019001A001B001C001D001E001F007C
:10684000200021002200230024002500260027002C
:10685000280029002A002B002C002D002E002F00DC
:1068600030003100000033003400350036003700BE
:10687000380039003A003B003C003D003E003F003C
:106880004000410042004300440045000000000079
:106890000000490000004B004C0000004E004F007B
:1068A000500051005200530054005500560057004C
:1068B000580059005A005B005C005D005E005F00FC
:1068C0006000610062006300000000000000000042
:1068D00000000000000000000000000000000000B8
:1068E00000000000000000000000000000000000A8
:1068F000E000E100E200E300E400E500E600F1A1D1
:106900000000000000000000010001000100010083
:10691000010001000100010046000100010001002A
:1069200001000100470048000100010001000100D2
:10693000010001000100010001000100010001004F
:10694000010001000100010001000100010001003F
:10695000010001000100010001000100010001002F
:106960000100010000000100010001000100010020
:10697000010001000100010001000100010001000F
:106980000100010001000100010001000000000001
:106990000000010000004A00010000004D004D0011
:1069A0004A004E004B0001000100010001000100FF
:1069B00001000100010001000100010001000100CF
:1069C00001000100010001000000000000000000C3
:1069D00000000000000000000000000000000000B7
:1069E00000000000000000000000000000000000A7
:1069F000010001000100010065000100010001002B
:00000001FF
